:100026006997FE013496EF93FF933196FA93EA931C
:1000360014E11A9317EF41221FEB412211E02ADF48
:100046000F931F9310E01F9310E01F9310E21F936E
:10005600E89445F84CD914E11F9318810F91011BC0
:10006600102FFF91EF9110832396FE0134961FEB1C
:10007600412220DCA801B901A0E0B0E0E0E8F4E408
:10008600E89441F8DEDA3B832A83198308833B81AF
:100096002A81198108810F931F932F933F937F9194
:1000A6006F915F914F91A0E0B0E0E0EAF0E4E89450
:1000B60041F855DA3B832A83198308833B812A81D9
:1000C6001981088108956997FE013496EF93FF938D
:1000D6003196FA93EA9314E11A9317EF41221FEB34
:1000E600412213E0D7DE0F931F9310E01F9310E019
:1000F6001F9310E21F93E89445F8F9D814E11F9373
:1001060018810F91011B102FFF91EF9110832396F9
:10011600FE0134961FEB4122CDDBA801B901A0E018
:10012600B0E0E0E8F4E4E89441F88BDA3B832A8314
:10013600198308833B812A81198108810F931F93B4
:100146002F933F937F916F915F914F91AAE0B7ED07
:10015600EBE6F1E4E89441F802DA3B832A8319835B
:1001660008833B812A811981088108956997FE01D8
:100176003496EF93FF933196FA93EA9314E11A9328
:1001860017EF41221FEB412212E084DE0F931F93EB
:1001960010E01F9310E01F9310E21F93E89445F8B8
:1001A600A6D814E11F9318810F91011B102FFF9100
:1001B600EF9110832396FE0134961FEB41227ADBE2
:1001C600A801B901A0E0B0E0E0E8F4E4E89441F861
:1001D60038DA3B832A83198308833B812A81198174
:1001E60008810F931F932F933F937F916F915F9198
:1001F6004F91A6E6B6EEEDECF2E4E89441F8AFD9FD
:100206003B832A83198308833B812A8119810881CC
:1002160008951127B1991FEF1095112309F401C014
:1002260001C0F7CF10E004E6FAD71127B1991FEF06
:10023600112309F401C001C0F8CF089511E017BBDE
:1002460013E018BB10E214BB10E015BB10E811BB9D
:1002560010E812BB10E8412A7894C1D7CF93DF93F8
:1002660010E01A9310E01A93A4D7DF91CF91CF93A1
:10027600DF9318E0412A07E218E01A930A93E6E2B0
:10028600FFE1B591BB2309F004D8DF91CF91CF935D
:10029600DF9310E01A9311E01A938BD7DF91CF9179
:1002A600CF93DF9318E0412A07E218E01A930A93E6
:1002B600E6E3FFE1B591BB2309F0EBD7DF91CF91E0
:1002C60017E000EDACD710E010936800C098979A3D
:1002D60086D7CF93DF9310E01A9310E01A9369D76D
:1002E600DF91CF91CF93DF9318E0412A07E218E020
:1002F6001A930A93E5E4FFE1B591BB2309F0C9D748
:10030600DF91CF91CF93DF9310E01A9311E01A9308
:1003160050D7DF91CF91CF93DF9318E0412A07E2C0
:1003260018E01A930A93E6E5FFE1B591BB2309F0BD
:10033600B0D7DF91CF916DDFC09A51D700E010E0C2
:1003460020E030E000936A0010936B0020936C006D
:1003560030936D0000E010E020E030E00093720082
:1003660010937300209374003093750000E010E042
:1003760020E030E000937600109377002093780019
:100386003093790010E000E0009380001093810024
:1003960010E01093680010916800139510936800A0
:1003A600A0918000B09181001196A0938000B09337
:1003B600810010E004E633D700E010E020E030E0F2
:1003C60000938A0010938B0020938C0030938D004D
:1003D60000918A0010918B0020918C0030918D0045
:1003E6000F931F932F933F93CF93DF9319DEDF91E4
:1003F600CF91E89441F8C9D900938A0010938B00F5
:1004060020938C0030938D0000918A0010918B0010
:1004160020918C0030918D0000936E0010936F0038
:10042600209370003093710000E010E020E030E08F
:1004360000938A0010938B0020938C0030938D00DC
:1004460000918A0010918B0020918C0030918D00D4
:100456000F931F932F933F93CF93DF9334DEDF9158
:10046600CF91E89441F891D900938A0010938B00BC
:1004760020938C0030938D0000918A0010918B00A0
:1004860020918C0030918D000093720010937300C0
:1004960020937400309375000091720010917300E0
:1004A60020917400309175000F931F932F933F9303
:1004B60000916E0010916F002091700030917100D4
:1004C600E89441F855D90093720010937300209375
:1004D60074003093750000E010E020E030E00093F7
:1004E6008A0010938B0020938C0030938D0000912E
:1004F6008A0010918B0020918C0030918D000F9313
:100506001F932F933F93CF93DF9330DEDF91CF91ED
:10051600E89441F83AD900938A0010938B0020930F
:100526008C0030938D0000918A0010918B002091F1
:100536008C0030918D000093760010937700209305
:100546007800309379000091760010917700209121
:100556007800309179000F931F932F933F9300916A
:100566006E0010916F002091700030917100E89438
:1005760041F8FED800937600109377002093780018
:100586003093790000916E0010916F0020917000F9
:1005960030917100A801B901A0E0B0E0EBEEF3E400
:1005A600E89441F84ED80F931F932F933F937F9172
:1005B6006F915F914F91A0E0B0E0EAE7F4E4E89430
:1005C60041F8CDD700936A0010936B0020936C001E
:1005D60030936D000091760010917700209178009D
:1005E600309179000F931F932F933F930DEC1CECE2
:1005F6002CE43DE3FF91EF91BF91AF91689442F8EF
:1006060055274CD7552339F00AF41AF09894889454
:1006160002C0989408941FEF08F011271F930091C9
:100626006A0010916B0020916C0030916D000F9361
:100636001F932F933F9300E010E020EA30E4FF91F0
:10064600EF91BF91AF91689442F8552727D755236C
:1006560039F00AF41AF09894889402C09894089491
:1006660010E011F008F01FEF0F911023112309F489
:1006760034C0B5D5CF93DF9310E01A9310E01A93E8
:1006860098D5DF91CF91CF93DF9318E0412A07E207
:1006960018E01A930A93E4E6FFE1B591BB2309F04B
:1006A600F8D5DF91CF91CF93DF9310E01A9311E045
:1006B6001A937FD5DF91CF91CF93DF9318E0412A2C
:1006C60007E218E01A930A93E2E7FFE1B591BB232C
:1006D60009F0DFD5DF91CF917CC3009176001091B0
:1006E600770020917800309179000F931F932F9314
:1006F6003F9300E010E028EC32E4FF91EF91BF91C8
:10070600AF91689442F85527C9D6552339F00AF4B3
:100716001AF09894889402C09894089410E011F006
:1007260008F01FEF112309F45BC000916A001091D5
:100736006B0020916C0030916D000F931F932F93E7
:100746003F9300E010E020E03FE3FF91EF91BF917F
:10075600AF91689442F85527A1D6552339F00AF48B
:100766001AF09894889402C0989408941FEF08F0A1
:100776001127112309F434C032D5CF93DF9310E04B
:100786001A9310E01A9315D5DF91CF91CF93DF938B
:1007960018E0412A07E218E01A930A93E0E8FFE11D
:1007A600B591BB2309F075D5DF91CF91CF93DF9338
:1007B60010E01A9311E01A93FCD4DF91CF91CF93F6
:1007C600DF9318E0412A07E218E01A930A93E1E959
:1007D600FFE1B591BB2309F05CD5DF91CF91F9C25A
:1007E6000091800010918100A0E81A27103809F4C2
:1007F600013010E009F41FEF112309F453C00091F2
:10080600720010917300209174003091750000936E
:10081600820010938300209384003093850000911A
:100826006A0010916B0020916C0030916D0000936E
:1008360086001093870020938800309389000091EA
:1008460086001091870020918800309189000F93CF
:100856001F932F933F9300E010E020E030E0FF91DC
:10086600EF91BF91AF91689442F8552717D655235B
:1008760039F00AF41AF09894889402C0989408946F
:1008860010E009F41FEF112309F40CC00DEC1CEC69
:100896002CE43DE3009386001093870020938800A4
:1008A600309389000091800010918100A0E81A27FA
:1008B600103809F4033010E009F41FEF1F9300917C
:1008C60072001091730020917400309175000F939F
:1008D6001F932F933F930DEC1CEC2CE43DE3FF910B
:1008E600EF91BF91AF91689442F85527D7D555231C
:1008F60039F00AF41AF09894889402C098940894EF
:1009060010E011F008F01FEF0F911023112309F4E6
:100916008FC0009172001091730020917400309185
:1009260075000F931F932F933F93009186001091AC
:1009360087002091880030918900E89441F805D617
:1009460000938A0010938B0020938C0030938D00C7
:1009560000916A0010916B0020916C0030916D003F
:100966000F931F932F933F93009182001091830062
:100976002091840030918500E89441F8E6D50093F3
:100986008E0010938F002093900030939100009179
:100996008E0010918F0020919000309191000F935E
:1009A6001F932F933F9300918A0010918B00209103
:1009B6008C0030918D00E89441F8DAD6E89441F83D
:1009C6003F770F931F932F933F930DEC1CEC2CEC6A
:1009D6003DE3FF91EF91BF91AF91689442F855279F
:1009E6005DD5552339F00AF41AF09894889402C01C
:1009F600989408941FEF08F01127112309F418C0E2
:100A0600EED3CF93DF9318E01A9310E01A93D1D365
:100A1600DF91CF911FE318D3CF93DF9318E01A939A
:100A260011E01A93C6D3DF91CF911FE30DD3D1C145
:100A3600009176001091770020917800309179002E
:100A46000F931F932F933F9300E010E020EA31E4C9
:100A5600FF91EF91BF91AF91689442F855271ED54B
:100A6600552339F00AF41AF09894889402C09894A1
:100A7600089410E011F008F01FEF112309F40DC0DF
:100A860000E010E020EA30E4009392001093930017
:100A960020939400309395000CC000E010E020E213
:100AA60031E40093920010939300209394003093C6
:100AB6009500009176001091770020917800309192
:100AC60079000F931F932F933F9300E010E020EFE0
:100AD60031E4FF91EF91BF91AF91689442F85527A9
:100AE600DDD4552339F00AF41AF09894889402C09C
:100AF6009894089410E011F008F01FEF112309F400
:100B060001C097986CD3CF93DF9310E01A9310E04F
:100B16001A934FD3DF91CF91009176001091770011
:100B260020917800309179000F931F932F933F9374
:100B36000AE919E929E131E4FF91EF91BF91AF91FB
:100B4600689442F85527AAD4552339F00AF41AF0C6
:100B56009894889402C0989408941FEF08F011277F
:100B6600112309F42BC0EAE7F0E0EF93FF933196E7
:100B7600FA93EA9315E01A9317EF41221FEB4122ED
:100B860000917200109173002091740030917500ED
:100B96000F931F932F933F9310E01F9317E01F931C
:100BA60010E21F9396D715E01F9318810F91011B32
:100BB600102FFF91EF91108323962AC0EAE7F0E009
:100BC600EF93FF933196FA93EA9315E01A9317EF92
:100BD60041221FEB4122009176001091770020916F
:100BE6007800309179000F931F932F933F9310E075
:100BF6001F9317E01F9310E21F936BD715E01F9307
:100C060018810F91011B102FFF91EF9110832396EE
:100C1600EAE7F0E0EF93FF933196FA93EA9315E053
:100C26001A9317EF41221FEB4122EAE7F0E0EF9318
:100C3600FF9311E01F9315E00F91FF91EF9116D3EB
:100C460015E01F9318810F91011B102FFF91EF9153
:100C560010832396CF93DF9318E0412A07E218E02A
:100C66001A930A93E2EAFFE1B591BB2309F011D387
:100C7600EAE7F0E013D3E8EAFFE1B591BB2309F018
:100C860008D3DF91CF91CF93DF9310E01A9311E051
:100C96001A938FD2DF91CF91EAE7F0E0EF93FF93BB
:100CA6003196FA93EA9315E01A9317EF41221FEB58
:100CB600412200916A0010916B0020916C003091E6
:100CC6006D000F931F932F933F9310E01F9317E030
:100CD6001F9310E21F93FDD615E01F9318810F9105
:100CE600011B102FFF91EF9110832396EAE7F0E0A6
:100CF600EF93FF933196FA93EA9315E01A9317EF61
:100D060041221FEB4122EAE7F0E0EF93FF9311E067
:100D16001F9315E00F91FF91EF91A8D215E01F9355
:100D260018810F91011B102FFF91EF9110832396CD
:100D3600CF93DF9318E0412A07E218E01A930A934B
:100D4600EBEAFFE1B591BB2309F0A3D2EAE7F0E0B5
:100D5600A5D2E1EBFFE1B591BB2309F09AD2DF9171
:100D6600CF9110916800103510E011F008F01FEFD8
:100D7600112309F401C02DC000916A0010916B0087
:100D860020916C0030916D000F931F932F933F932A
:100D9600009192001091930020919400309195005B
:100DA600FF91EF91BF91AF91689442F8552776D3A2
:100DB600552339F00AF41AF09894889402C098944E
:100DC600089410E008F01FEF112309F401C001C0D8
:100DD600E2CA10E010936800CF93DF93C7D9DF9182
:100DE600CF910F931F932F933F9300E010E020EFD6
:100DF60031E4FF91EF91BF91AF91689442F8552786
:100E06004DD3552339F00AF41AF09894889402C009
:100E16009894089410E011F008F01FEF112309F4DC
:100E260001C0DACF979AC098F4D952CAFFCFF89486
:100E360011E00BE01EBF0DBF1127E9E0F0E0A6E0D0
:100E4600B0E03196319711F01D93FCCF1127E0E009
:100E5600F4E0A0E6B0E03196319711F01D93FCCF97
:100E6600CFE6D1E0F8941FE7412240D814E610936C
:100E7600600012BF15E013BF11E019BF7724882464
:100E86009924B99A11271DBD1CBD1BBD1ABD13E8B7
:100E96001FBD13E010934E00112717B917EC16B9B2
:100EA600112712BB1FE711BB13E012BB00E111278C
:100EB600B6D112B3106112BB00000000000012B3DD
:100EC6001F7E12BB05E01127AAD112B3106112BB17
:100ED60000000000000012B31F7E12BB01E01127C4
:100EE6009ED112B3106112BB00000000000012B3C5
:100EF6001F7E12BB12E012BB01E0112790D112B384
:100F0600106112BB00000000000012B31F7E12BB6E
:100F160001E0112784D112B3106112BB000000005A
:100F2600000012B31F7E12BB18E012BB01E01127AE
:100F360076D112B3106112BB00000000000012B39C
:100F46001F7E12BB1CE08BD011E089D016E087D043
:100F560014B3106214BB15B31F7D15BB11E015BD8C
:100F660019B7106419BF10E614BD4424552466C988
:100F7600EF93FF930F931F931FB71F93109160007A
:100F860002B7100F12BF1FE7412204B115B11F931C
:100F9600E7B1E770EF93F0916700F17041F4E395E4
:100FA600E33008F0EE27F7B1F87FEF2BE7B91F9192
:100FB600110FE1E6F0E0E10F08F4F3951F910083CD
:100FC600118316B30FEF1027012F1725782C8122D6
:100FD60010951023812A10E0709471261825172188
:100FE600912A702E10E8412A369A1F911FBF1F9131
:100FF6000F91FF91EF911895EF93FF930F931F9326
:101006001FB71F9310E614BD2F9310916900139517
:10101600153609F41127109369002227E8E6F0E057
:101026000191002329F0053611F0011708F020621E
:1010360015B31F7D122B15BB2F911F911FBF1F913B
:101046000F91FF91EF9118951F9354D011B31F671D
:1010560011BB12B31F7E1079106212BB09C01F9319
:1010660049D011B31F6711BB12B31F7E107912BB93
:101076001F911F9312951F7002B3012B02BB1F9184
:10108600000000000000000000000000006102BB3C
:1010960000000000000000000000000002B30F7E08
:1010A60002BB0000000000000000000000001F70EE
:1010B60002B3007F012B02BB00000000000000000D
:1010C60000000000006102BB0000000000000000FC
:1010D6000000000012B31F7E12BB08950BD011B39F
:1010E600107F11BB12B31F7E107F106612BBE894EF
:1010F60044F817C0E0E8F2E0689444F802C0E894C7
:1011060044F811B3107F106311BB12B31F7E1F7911
:1011160012BB000000000000000000000000106488
:1011260012BB00000000000000000000000012B327
:10113600106112BB0000000000000000000000006B
:1011460000B30295007F12B31F7E12BB00000000A1
:10115600000000000000000012B3106112BB000086
:101166000000000000000000000010B31F70102BEC
:1011760002B30F7E007F02BB44FA0EF0089531974A
:1011860019F0111F70F208951FEF08951FEF0FEF6A
:1011960006C0FF91EF911F910F91EF93FF931123DB
:1011A60011F41CE001C01DE0002309F0126057DFB6
:1011B600089518810981103011F410E80DC011301E
:1011C60011F410EC09C0123011F410E905C0133007
:1011D60011F410ED01C010E8100F41DF089511E081
:1011E6003EDF0895103011F410E80DC0113011F4EF
:1011F60010EC09C0123011F410E905C0133011F4D7
:1012060010ED01C008951F932ADF10E11F9310E22D
:101216001BDF1F911A95D1F71F9121DF0895A801B1
:1012260011274117510749F00AE71CE00150104009
:101236000000E1F741505040B9F70895112331F00D
:1012460006E20A950000E9F71A95D1F708952150AC
:10125600304018F011911D93FACF0895B12F1191D6
:10126600112319F079D5BA95D1F70895112381F094
:10127600B081BB2369F0B01B58F0B395AA27E00FE5
:10128600FA1FB11708F0B12F119166D5BA95E1F79B
:101296000895159161D5BA95E1F708951191112335
:1012A60029F0B12F119158D5BA95E1F708950D910E
:1012B6001D9152D53A9511F41EE24ED50A95C1F705
:1012C600FF91EF9108810083098101830A810283DE
:1012D600EF010895E881EE2311F4112339F0E39527
:1012E600E883FF27EC0FFD1F106310830895BF915D
:1012F600AF91EF914F915F911F910F91AF93BF9374
:10130600CF93DF932997AA27A8835F834887EF9314
:10131600E2E1FFE1D801E89442F845FA16F417FD38
:1013260042F864E0259135913296EF93FF935DD5AF
:10133600DF01102F11230AF41195CCDFFF91EF91F5
:101346006A9581F71A2FC6DF5F91FF91EF91EF93B0
:10135600FF93DE0128853F8100C00881002321F428
:101366000395088310E3198323970081088301817D
:10137600098302810A83332389F1222379F14C916F
:101386003A95431738F0342F321B42FA16F41DE211
:10139600E3D48DCF042F241714F0022F039542FABD
:1013A6000EF43A95152F031B019529F022F0D4D49B
:1013B6003A950A95E1F742FA16F41DE2CDD4321BAE
:1013C600241758F010E3C8D41EE2C6D43327241BD2
:1013D60021F010E3C1D42A95E1F769CF42FA16F459
:1013E6003A9542F00C91301B29F020F0152FB4D419
:1013F6003A95E9F742FA16F41DE2AED458CF6F9348
:101406007F93732F622F661F771F7F5738F47F9164
:101416006F91112700273327222708952068632F0D
:101426003327783148F47751719571F036952795C1
:10143600179507957A95F9CF775131F0000F111F5F
:10144600221F331F7A95F9CF67FF08C0015010405D
:101456002040304000951095309520957F916F91F2
:1014660008953F3C28F030E82227112700270895E9
:1014760037FD07C03F3428F03FE72FEF1FEF0FEF90
:10148600089537FFBCCF3F77BADF015010402040A8
:10149600304020953095109500950895432F4F23A1
:1014A600407837FF03C03F7747FF12C0F7FF03C0FE
:1014B600FF7747FF15C03F1758F091F42E1740F0FD
:1014C60079F41B1728F061F40A1710F049F40BC0E1
:1014D60047FD08C042FA16F08D019F01539503C0DF
:1014E60047FDF8CF5A95342B0895332339F4222338
:1014F60029F4112319F4002309F40895AA2745FEB7
:101506000CC0A32FA078332342F401501040204092
:1015160030402095309510950095B6E9332331F08B
:101526003695279517950795B395F8CF27FD06C0ED
:10153600000F111F221F331FBA95F8CF2F773B2FAD
:10154600369508F420683A2B0895D801F9011F91C1
:101556000F917F916F915F914F910F931F93FF238F
:1015660011F0772329F4002711272227332708951E
:101576003F2F37273078EE1FFF1F0894E795661F29
:10158600771F089467951127F70F111FFF57104013
:10159600112311F4FF3F40F0689441F830783E671C
:1015A6002FEF0FEF1FEF0895F13038F4332722277E
:1015B60000271127689441F808953F93FF93FF276A
:1015C60077279927882711240024769567955795BC
:1015D600479510E220F48A0F9B1F0E1E1F1E1794BC
:1015E60007949795879577956795579547951A9593
:1015F60089F727E1169407949795879577956795C8
:10160600579547952A95B1F7042F152F262F372F73
:10161600BF910F90332329F0369527951795079597
:10162600B395302D221FB69527953B2B0895D801EB
:10163600F9011F910F917F916F915F914F910F93D8
:101646001F933F2F37273078FF2341F4689441F8E2
:1016560030783E672FEF1FEF0FEF0895EE1FFF1F45
:101666000894E795661F771F08946795772329F4F2
:101676003327222711270027089511277F1B1040A3
:10168600F72F0EE7F00F0027101F112311F4FF3F6D
:1016960041F4689441F830783E672FEF0FEF1FEF63
:1016A6000895FF2339F4689441F833272227002749
:1016B600112708953F93FF93FF2788279927762FB1
:1016C600652F542F442710E32227332700241124A3
:1016D600222433248894881F991F441F551F661F90
:1016E600771F221F331F001C111C221C331C48F4B9
:1016F60000272A1B3B0B0E0A1F0A200A300A0894F1
:1017060019C000273016B0F071F4201698F059F47D
:101716001F1680F041F40E1668F029F43B1750F0BE
:1017260011F42A1738F000272A1B3B0B0E0A1F0A52
:10173600200A300A1A9510F0089401C0889459F6C8
:10174600881F991F441F551F661F771F082F192FC3
:10175600242F352FBF91332329F0369527951795DA
:101766000795B3953F91221FB69527953B2B089574
:10177600D801F9011F910F917F916F915F914F9160
:101786000F931F9310E8F1270AC0D801F9011F91A2
:101796000F917F916F915F914F910F931F931F2F21
:1017A6001F77072F0F77011790F041F46E1778F027
:1017B60029F45B1760F011F44A1748F08A019B017F
:1017C6005B2F4A2F7F2F6E2FD801F90102C08D01A2
:1017D6009F012F7720683327F7FF08C0015010407C
:1017E6002040304020953095109500951F939F2FEF
:1017F6008E2F881F991F872F062E001C881F152ED7
:10180600042E262E10E8212A3324192F181B112303
:1018160029F02694179407941A95FACF172F402D7E
:10182600512D622D732D17FF08C041505040604066
:10183600704040955095709560951F91040F151F47
:10184600261F371F37FF0AC0F0680150104020409E
:101856003040209530951095009501C0FF77832F75
:101866008F7779F03695279517950795939549F4CF
:101876001FEF0FEF2FEF3FE7F7FD3068689441F851
:10188600089527FD08C0992331F0000F111F221F6C
:10189600331F9A95F6CF392F99273695332331F092
:1018A60097952F77292BF7FD306808952227112762
:1018B60000270895E89441F83324222411270027AD
:1018C600332722272F93A0813196B1D0BAD0F0F0DA
:1018D6004B3219F43196AA95F9CF4D3239F44F911E
:1018E60040954F933196AA95ACD080F04E3229F4AC
:1018F6003196AA95A6D008F44AC04F9133242224E3
:1019060011270027689441F8089408959AD0D8F5CD
:1019160047D03196AA954423C9F333953196AA95B3
:1019260090D0D8F34E3229F48CD018F43196AA957B
:10193600FBCF453419F0453609F053C03196AA95C8
:1019460080D050F04D3219F04B3211F0D6CF2094A2
:101956003196AA9576D088F64053342E3196AA95BC
:1019660070D050F4532D550F550F530D550F40534E
:10197600450F342E463208F6432D22200AF44195AF
:10198600430F342F2EC04E32A1F63196AA9559D068
:1019960080F606D03196AA95442331F63A95F7CFCC
:1019A600822F712F602F000F111F221FA8F0000F2A
:1019B600111F221F88F0060F171F281F68F0000F3F
:1019C600111F221F48F0408140535527040F151F51
:1019D600251F10F044270895282F172F062F4FEFA5
:1019E60008954F913CD011F1332E3327E89441F8F6
:1019F600E89445F87ADD47FD3068232C3320B1F0B2
:101A06000AF4319422202AF0A0E0B0E0E0E2F1E40A
:101A160004C0ADECBCECECECFDE3402F512F622F83
:101A2600732FE89441F89BDD3A9461F70895AA2351
:101A360009F408954081403219F43196AA95F7CFFA
:101A46000895AA2319F444278894089540814033C1
:101A560020F04A3310F408940895889408953323A7
:101A660029F4222319F4112309F4002308955F931E
:101A7600B801C901AFE7B6E9E8E1FBE4689442F8CA
:101A860055270CDD8B019C015523CAF0C1F0A0E05F
:101A9600B4E2E4E7F9E4552701DD5523C2F0B9F0D5
:101AA6005F915A955F93A0E0B0E0E0E2F1E4462F43
:101AB600572F682F792FE89441F851DDD9CF5F91E0
:101AC60053955F93ADECBCECECECFDE3F0CF5F918E
:101AD60008955F914F91EF91AF91BF913F912F91F3
:101AE6001F910F914F935F93CF93DF9371E160E363
:101AF6006A937A95E9F700240882BE87AF87E88B58
:101B0600E89441F8732F7F777723A9F41F850EE2B7
:101B1600153449F41FEF1F8710E312D115E410D1D5
:101B260010E30ED1A8C010E30BD11EE209D110E3D9
:101B360007D1F7D0A0C0552733232AF43F771F9348
:101B46001DE2FED01F9193DF5F936F937F938F9378
:101B56009F9300E010E020E03FE34F85AE85585F9D
:101B66005830F4F45B3FE4F04534D1F0AA2309F48D
:101B7600451BA52F59E0541B5A1B92F019F450959A
:101B86005F870EC05A9561F05F93A801B901A0E086
:101B9600B0E0E0E2F1E4E89441F8E1DC5F91F2CFF5
:101BA600E89441F8F2DD5F9162DF5F93B801C90105
:101BB600221F331F8068315831953B5E04C08695DD
:101BC600779567953A95D9F7BF91A1E04F8545344A
:101BD60029F4B85F2B2F0AF4219509C027E0B85FD6
:101BE600B8302CF4BB3F1CF0BA95AB2FB2E0B25024
:101BF600AA2309F05AF410E3A3D01EE2A1D0AA2327
:101C060029F010E39DD02A95A395D9F7EAE0FFE1E4
:101C16003327059114913196C8953296601B710B46
:101C2600800910F03395FACF600F711F801D3A308E
:101C360014F031E0B39510E3130F82D0AA9511F496
:101C46001EE27ED02A950AF019F76BD0BB2399F0D5
:101C56001FEF1F8715E474D0BB231AF4B1951DE25C
:101C66006FD00AE01B2FB1D0112311F0106368D09A
:101C7600102F106365D0FF91EF91DE012F853E8511
:101C86002397008108830181098302810A832F3FFC
:101C960021F1332311F1222319F436D05C931DC0B0
:101CA60033D04C91321B3A95351B29F020F01B8915
:101CB60053D03A95E9F75C9321D01EE24DD01196A8
:101CC600451B4A9529F01D9147D02A9579F0F9CF01
:101CD60010E342D02A95E1F709C00C91301B29F098
:101CE60020F01B8939D03A95E9F708D0088100839E
:101CF600098101830A810283EF0108950D911D91E7
:101D06002BD00A95E1F70895AF93BF9355270D9110
:101D16001D911E3219F053950A95D1F7BF91AF91D7
:101D26000895E8811E2FE395FF27EC0FFD1F1A95F6
:101D360002910033E1F30E3209F0139518830895EA
:101D4600EF93FF93E881E395E883FF27EC0FFD1FF0
:101D56001083FF91EF910895EF93FF9343FAAEF04E
:101D66001F93E981FA811881112331F41F91689438
:101D760041F8FF91EF9108951A9518831F911193D9
:101D8600FA83E983FF91EF910895E881F9811F9322
:101D96000F932F933F93AF93BF936F937F934F937D
:101DA6005F9309955F914F917F916F91BF91AF912D
:101DB6003F912F910F911F91FF91EF9108953F91C0
:101DC6002F91012F1F912F933F93332729E0111F46
:101DD6002A9511F4032F0895331F301B18F4300F82
:101DE6008894F5CF0894F3CF9801552745FA96F4D1
:101DF6005B2F432F4B27E89447FF45F837FF04C076
:101E0600219509F43A953095B7FF04C0A19509F4D8
:101E1600BA95B095EE27FF1B11E1AA1FBB1F1A95B5
:101E260041F48D0145FA26F4019509F41A951095A9
:101E36000895EE1FFF1FE21BF30B20F4E20FF31FC2
:101E46008894EBCF0894E9CF1770E6EFFEE1002403
:101E5600E10FF01DC8951127082D002109F01095F6
:101E660008951770E6EFFEE10024E10FF01DC89516
:101E7600302D30951127092D002109F01095F89481
:101E8600092D0323902E47FC78940895112710936B
:101E960009000895112379F0143068F41A95110F8A
:101EA6000027E1E6F0E0E10FF01FF89401911081C0
:101EB60047FC78940895002711270895F894009117
:101EC60067001981112311F40E7F0BC00160188180
:101ED600112339F0143028F41A95F7B1F87F1F2B27
:101EE60017B90093670047FC7894089508951895EC
:101EF600010204081020408000CA9A3B00E1F50563
:101F06008096980040420F00A0860100102700002E
:101F1600E8030000640000000A0000000100000061
:101F26000F5A454E45524D455452452056312E3096
:101F36000E422E4C656272756E2030382F3034108A
:101F46005072657420706F7572206C616E63657275
:101F56000D756E65206D65737572652E2E2E0D439B
:101F66006F6D706F73616E7420656E200D636F7593
:101F760072742D636972637569741050617320649D
:101F86006520636F6D706F73616E74106F75205589
:101F96007A2074726F70206772616E6405557A20BC
:0F1FA6003D2002205605497A203D2003206D4141
:1000000019C778CF77CF76CFFAC774CF73CF72CFB7
:1000100071CFB1C76FCF6ECF6DCF6CCF6BCF6ACFC3
:0600200069CF68CF67CF35
:00000001FF
